:020000040000FA
:10000000B2017929A400360884003408C72084137B
:1000100000052C1C3406031920282408031D182869
:100020002A08FF3E031C21289630DF202A082128B9
:10003000240AFF3003192028240B20282B0821280C
:10004000AD09AD0C7429A501A400B3172730A30096
:10005000103036200330A300E8303620A30164308E
:100060003620A3010A30362024084128A2002508A2
:10007000A1002408A00042212008031DB313B31BD4
:100080000800303EA700061186118611831606115E
:10009000861186110F30860583122708B2186D2845
:1000A0003A30A100FC30ED203330A6008120103022
:1000B000A1006830ED2081206430EC202230A600C1
:1000C000812028306C200C306C2001306C200630F0
:1000D0006C20B21427086D283214A600321C7B282D
:1000E0008611033C031C802880200530A100DC30F1
:1000F000ED20031408003214FE3C03197429861500
:10010000321C321006150F3086052608F039860499
:100110000611A60E321881282C30EC20031408009A
:100120000830A6003708840035083319C220331D73
:10013000C420360884003409CB202608031974290A
:100140003318012136088400A10CA00C00083404E7
:10015000031C34068000AF20A60BA22874293708A0
:100160008400350880062008A2002108A300003082
:10017000A1000C30ED202208A0002308A1003508C2
:10018000800608008004CA28FF3A8005CB2884171F
:1001900080047429FF3A84178005742983169B0014
:1001A0001C141A08742983169A001C1555309D00DA
:1001B000AA309D009C149C18DB281C117429A301F3
:1001C000A200FF30A207031CA307031C74290330FD
:1001D000A100DF30ED20E128A101E83EA000A10947
:1001E000FC30031CF628A0070318F328A0076400BE
:1001F000A10FF3282018FC28A01C002900000029CA
:100200000800A201A3010829A10CA00CA20DA30DB6
:10021000FF3E031804292308A1002208A000742926
:10022000A20003302029A101A301A200013020294E
:10023000A20006302029A20004302029A2000530A7
:10024000A80023082102031D2729220820020430C8
:1002500003180130031902302805031DFF307429EB
:100260000404031DFF307429A2002008A6002408FE
:10027000A0002608A4002108A6002508A100260841
:10028000A5004429A501A4011030A600210DA40D4C
:10029000A50D2208A4022308031C230FA50203189E
:1002A00058292208A40723080318230FA5070310C1
:1002B000A00DA10DA60B4629200874291030A80016
:1002C000A101A001A70CA60C031C6C292208A00701
:1002D00023080318230FA107A10CA00CA50CA40C44
:1002E000A80B622924087429831303138312640062
:1002F000080083160515851505148514831207302B
:100300009F0064006430DF20FE3042200130422034
:10031000503042204C3042204C304220203042208D
:10032000303042202E30422036304220623042208F
:10033000FE304220C0304220443042204C30422027
:10034000313042204D304220463042204B30422056
:100350000530A300DC30E020DC01BC01BD01DB0185
:10036000C630B800B9019F260130DB001923F72100
:10037000D2220530B6000130B400AC01FF30AA0033
:10038000AB010130AD0058080220D8000318C9297C
:10039000D429DC0A640005305C02031CD029DC018E
:1003A000FE3042200C30422064005C08003C031DFB
:1003B000DB293C2BF62964005C08013C031DE22983
:1003C0006A2DF62964005C08023C031DE9293F2FD1
:1003D000F62964005C08033C031DF029C52BF629AF
:1003E00064005C08043C031DF629D52CB929403073
:1003F0005402C8000730031C013E5502C9004808DA
:10040000A6004908A700A2010130A3005E21BA009E
:100410002508BB000330A300E8303421C2002108C6
:10042000C3004808A0004908A100E830A20003303A
:10043000A3004221D0002108D1005008A600510895
:10044000A700E830A2000330A3005E21D0002508F9
:10045000D10050084802C6005108031C013E490261
:10046000C7004608A6004708A7004030A200A30125
:100470005E21C6002508C7004608A0004708A10065
:10048000E830A2000330A3004221D0002108D100AF
:100490005008A6005108A700E830A2000330A300CE
:1004A0005E21D0002508D1005008C6025108031C67
:1004B000013EC7024608A6004708A7000430A20074
:1004C000A3015E21C6002508C7004608A000470812
:1004D000A100E830A2000330A3004221D00021088F
:1004E000D1005008A6005108A700E830A200033050
:1004F000A3005E21D0002508D10050084602BE00AE
:100500005108031C013E4702BF0064005A1CD12A57
:100510006400DA1CB22A3E084002BE003F08031CF9
:10052000013E4102BF0042084402C2004308031CCE
:10053000013E4502C3003E08A0003F08A100033071
:10054000A300E7301821031DB12A1730BE02FC308A
:10055000031C013EBF020130C2020030031C013EF9
:10056000C302D12A4008BE0741080318013EBF0755
:100570004408C20745080318013EC3073E08A0000F
:100580003F08A1000330A300E7301821031DD12A42
:10059000E830BE020330031C013EBF02C20A031949
:1005A000C30A0800FE304220C03042204208A000AA
:1005B0004308A1002730A30010301021031DEE2AAC
:1005C000203042204208A0004308A1000330A300CD
:1005D000E8301021031DEE2A203042204308A500F8
:1005E000420824202E3042203E08A0003F08A100EF
:1005F000A30164301021031D0A2B303042203E0835
:10060000A0003F08A100A3010A301021031D0A2BFE
:10061000303042203F08A5003E08242020304220F0
:100620004D304220483042207A3042202030422053
:1006300008000516831605120C308312EC200630D4
:10064000B6001030B4000630B7002030B5000130DD
:10065000B3000530A000A10190205508A000A10121
:1006600090205408A000A10190200C30EC2005122D
:1006700083160512831208001923F721FE30422049
:10068000013042202030422020304220563042208B
:10069000463042204F304220D2220530B60004308E
:1006A000B400AC01FE30AA00AB010130AD00560829
:1006B0000220D60003187B2B0530B6000830B400AA
:1006C000AC01FE30AA00AB010130AD00570802209A
:1006D000D7000318982B0530B6000130B400AC01E8
:1006E000FF30AA00AB010130AD0058080220D8004D
:1006F0000318C9294D2B6400DA1C7F2B9C2BD40ACC
:100700000319D50A64008518892B2630D4070318ED
:10071000D50A5408A0005508A1002630A30099303E
:100720001821031D972BF830D4001430D500B92BB5
:100730006400DA1C9C2B7F2B0130D4020030031C98
:10074000013ED50264008518AB2B2630D402003060
:10075000031C013ED5025408A0005508A100143026
:10076000A300F8301021031DB92B9930D400263096
:10077000D50083169B0183125508D32083160130C0
:100780009B0083125408D3203C2BFE3042200130C2
:10079000422020304220203042204C3042206F3016
:1007A00042202030422051304220523042204730F7
:1007B00042204408C2004508C3004008BE0041086A
:1007C000BF00D222FE30422038084220FE304220B4
:1007D0000E3042200530B6000430B400AC01FE30CB
:1007E000AA00AB010130AD0056080220D600031864
:1007F000562C0530B6000830B400AC01FE30AA001B
:10080000AB010130AD0057080220D70003187C2C43
:100810000530B6000130B400AC01FF30AA00AB01D6
:100820000130AD0058080220D8000318C92905304E
:10083000B6000230B400AC01FF30AA00AB010130B9
:10084000AD0059080220D9000318272CEA2B3C08D8
:10085000A6003D08A7000A30A200A3015E21BC004B
:100860002508BD000130B8020030031C013EB9026A
:10087000A001A1013D08A3003C081E21031D462C38
:100880000130BC00BD01C430B800B9011030A00077
:100890002730A1003D08A3003C081E21031D552C54
:1008A000BC01BD01C630B800B901C52BA001A10132
:1008B0003D08A3003C081E21031D662C7D30C007A7
:1008C0000318C10AC630B800B9016C2C3C08C40733
:1008D0003D080318013EC507E830A0000330A10021
:1008E0004108A30040081E21031D7B2CC001C1014B
:1008F000C40A0319C50AB42CA001A1013D08A30034
:100900003C081E21031D8E2C7D30C0020030031CCC
:10091000013EC102C630B800B901942C3C08C402A3
:100920003D08031C013EC5024008A0004108A1008B
:100930000330A300E8301B21031DA82C6B30C0003E
:100940000330C1000130C4020030031C013EC50267
:100950004408A0004508A100C330A300503018216E
:10096000031DB42CC401C5014408C2004508C300DE
:100970004008BE004108BF00831602309B0083126E
:100980004508D320831603309B0083124408D320EC
:10099000831604309B0083124108D3208316053050
:1009A0009B0083124008D320C52BFE30422001302B
:1009B000422020304220203042204C3042206F30F4
:1009C000422020304220413042206E3042202F30E1
:1009D0004220413042207530422073304220FE30A8
:1009E0004220C030422064005A18032D4C3042206F
:1009F0004F304220203042204130422055304220AA
:100A0000533042201F2D6400DA18132D413042204C
:100A10004E30422020304220283042202B304220CD
:100A2000293042201F2D413042204E3042202030BC
:100A30004220283042202D304220293042200530EB
:100A4000B6000430B400AC01FF30AA00AB010130A5
:100A5000AD0056080220D60003185C2D0530B60004
:100A60000830B400AC01FF30AA00AB010130AD008A
:100A700057080220D70003185F2D0530B60001305B
:100A8000B400AC01FF30AA00AB010130AD00580842
:100A90000220D8000318C9290530B6000230B4007E
:100AA000AC01FF30AA00AB010130AD0059080220B3
:100AB000D9000318622D1F2DDA105A14632DDA1491
:100AC0005A14632D5A10831606309B0083125A085D
:100AD000D320D52C5408CE005508CF004408CC00B4
:100AE0004508CD004008CA004108CB005A08DD0087
:100AF000FE3042200130422020304220203042206F
:100B0000533042206130422076304220653042200E
:100B1000203042205B0823209F26F721D222053077
:100B2000B6000430B400AC01FF30AA00AB010130C4
:100B3000AD0056080220D6000318CC2D0530B600B3
:100B40000830B400AC01FF30AA00AB010130AD00A9
:100B500057080220D7000318D52D0530B600013004
:100B6000B400AC01FF30AA00AB010130AD00580861
:100B70000220D8000318EF2D0530B6000230B40073
:100B8000AC01FF30AA00AB010130AD0059080220D2
:100B9000D9000318FE2D8F2DDB0A640012305B0292
:100BA000031CD42D0130DB00782DDB035B08003CF7
:100BB000031DFF30FF3AD0005B08A0001130132165
:100BC000D2005008840052083021D200D3006400C3
:100BD000520853040319EE2D1130DB00782D4E0816
:100BE000D4004F08D5004C08C4004D08C5004A0881
:100BF000C0004B08C1005D08DA00C9294E08D400C6
:100C00004F08D5004C08C4004D08C5004A08C00074
:100C10004B08C1005D08DA005B08A600A701073099
:100C2000A200A3015E21D0002508D1000030D0072A
:100C30000318D10A500883169B0083125508D3204D
:100C40005B08A600A7010730A200A3015E21D00027
:100C50002508D100D00A0319D10A500883169B0039
:100C600083125408D3205B08A600A7010730A20016
:100C7000A3015E21D0002508D1000230D00703185F
:100C8000D10A500883169B0083124508D3205B08C5
:100C9000A600A7010730A200A3015E21D00025080D
:100CA000D1000330D0070318D10A500883169B00E7
:100CB00083124408D3205B08A600A7010730A200D6
:100CC000A3015E21D0002508D1000430D00703180D
:100CD000D10A500883169B0083124108D3205B0879
:100CE000A600A7010730A200A3015E21D0002508BD
:100CF000D1000530D0070318D10A500883169B0095
:100D000083124008D3205B08A600A7010730A20089
:100D1000A3015E21D0002508D1000630D0070318BA
:100D2000D10A500883169B0083125A08D320DC0195
:100D3000F721D2220530A300DC30E0203C2B5B08F9
:100D4000A600A7010730A200A3015E21D00025085C
:100D5000D1000030D0070318D10A5008CE20D500AA
:100D60005B08A600A7010730A200A3015E21D00006
:100D70002508D100D00A0319D10A5008CE20D4008A
:100D80005B08A600A7010730A200A3015E21D000E6
:100D90002508D1000230D0070318D10A5008CE2010
:100DA000C5005B08A600A7010730A200A3015E21D1
:100DB000D0002508D1000330D0070318D10A50080D
:100DC000CE20C4005B08A600A7010730A200A30143
:100DD0005E21D0002508D1000430D0070318D10AC5
:100DE0005008CE20C1005B08A600A7010730A20072
:100DF000A3015E21D0002508D1000530D0070318DB
:100E0000D10A5008CE20C0005B08A600A701073019
:100E1000A200A3015E21D0002508D1000630D00732
:100E20000318D10A5008CE20DA0083169B018312E2
:100E30005508D320831601309B0083125408D32019
:100E4000831602309B0083124508D320831603309B
:100E50009B0083124408D320831604309B00831226
:100E60004108D320831605309B0083124008D3200D
:100E7000831606309B0083125A08D32008005408BA
:100E8000CE005508CF004408CC004508CD004008EE
:100E9000CA004108CB005A08DD00FE304220013074
:100EA000422020304220203042204D304220453028
:100EB00042204D304220203042205B0823209F26D4
:100EC000F7211923D2220530B6000430B400AC015A
:100ED000FF30AA00AB010130AD0056080220D60059
:100EE0000318A02F0530B6000830B400AC01FF3065
:100EF000AA00AB010130AD0057080220D70003184B
:100F0000A92F0530B6000130B400AC01FF30AA00B3
:100F1000AB010130AD0058080220D8000318B22FF1
:100F20000530B6000230B400AC01FF30AA00AB01BE
:100F30000130AD0059080220D9000318C12F632FDA
:100F4000DB0A640012305B02031CA82F0130DB00B7
:100F50004D2FDB03640001305B020318B12F113009
:100F6000DB004D2F4E08D4004F08D5004C08C400BC
:100F70004D08C5004A08C0004B08C1005D08DA00F2
:080F8000C9299F26DC013C2B6E
:02400E00703F01
:104200001900A00023002800000000000000190091
:10421000A000230028000000000000001900A000FA
:10422000230028000000000000001900A000230067
:1042300028000000000000001900A0002300280052
:104240000000000000001900A0002300280000006A
:10425000000000001900A00023002800000000005A
:1042600000001900A000230028000000000000004A
:104270001900A00023002800000000000000190021
:10428000A000230028000000000000001900A0008A
:10429000230028000000000000001900A0002300F7
:1042A00028000000000000001900A00023002800E2
:1042B0000000000000001900A000230028000000FA
:1042C000000000001900A0002300280000000000EA
:1042D00000001900A00023002800000000000000DA
:1042E0001900A000230028000000000000001900B1
:0C42F000A00023002800000000000000D7
:00000001FF
